:1000000031C029CD3DCD48C071C046C045C044C0B7
:1000100043C042C041C0FBC03FC03EC03DC03CC029
:100020003BC03AC039C089CAA5CAC3CAD2CAFACA33
:100030001ACBD6CBD5CBD4CBD3CB29CB32CB43CB5E
:1000400056CBCECBCDCBCCCBCBCBCACBC9CB55CBE8
:1000500061CB7CCBC5CBC4CBC3CBC2CBC1CBC0CBDC
:10006000BFCB92CB11241FBECFE5D4E0DEBFCDBF06
:1000700011E0A0E6B0E0E8E4FBE102C005900D92DB
:10008000A634B107D9F713E0A6E4B1E001C01D9290
:10009000AA3CB107E1F7FCCBB3CF9C012150304023
:1000A0008FEF2F3F380729F088EC9AE00197F1F79E
:1000B000F5CF08959C01215030408FEF2F3F380736
:1000C00029F083E090E00197F1F7F5CF089589B723
:1000D000806489BF83E684BD85B5816085BD85B5B3
:1000E000826085BD85B5846085BD08951F920F929D
:1000F0000FB60F9211241F932F933F934F935F934B
:100100006F937F938F939F93AF93BF93CF93DF931F
:10011000EF93FF93CDE6D1E013E08881813089F53C
:100120008B819C81AD81BE810197A109B1098B832F
:100130009C83AD83BE838B819C81AD81BE81009702
:10014000A105B105F1F489819A81892BD1F08981CA
:100150009A818F5F9F4F29F089819A8101979A83B5
:10016000898389819A81892B09F418828F819885E6
:10017000A985BA858B839C83AD83BE83EB85FC8583
:10018000099511502D9617FFC8CF83E684BDFF91C6
:10019000EF91DF91CF91BF91AF919F918F917F911F
:1001A0006F915F914F913F912F911F910F900FBED3
:1001B0000F901F9018950F931F93DB01BA01A901AF
:1001C000282F33278DE090E0289FF001299FF00D24
:1001D000389FF00D1124E359FE4FB283A18343836E
:1001E000548365837683478350876187728714873A
:1001F000038781E080831F910F91089588E089B97A
:1002000088E18AB908955D9BFECF8CB908951F924D
:100210000F920FB60F9211248F93EF93FF9380915B
:100220006C01E82FFF27EA54FE4F8CB18083809148
:100230006C018F5F80936C0180916C01843110F0B0
:1002400010926C01FF91EF918F910F900FBE0F9064
:100250001F9018951F9380916C01882369F010916D
:100260006C0185E090E019DF80916C01811721F02D
:1002700080916C01882399F71F9108951F93182F7F
:1002800082958F70E82FFF27EF59FF4F8081BBDFEA
:100290001F70E12FFF27EF59FF4F8081B4DF1F91BF
:1002A0000895CF93DF93EC018881882329F0899109
:1002B000AADF88818823D9F7DF91CF910895EF9243
:1002C000FF920F931F937C0100E117E2B80114DC49
:1002D000CB01805D98DFC701B8010EDC08EE13E0AA
:1002E000B8010ADCCB01805D8EDFC701B80104DCF8
:1002F00004E610E0B80100DCCB01805D84DFC701BB
:10030000B801FADB0AE010E0B801F6DBCB01805D52
:100310007ADFC701B801F0DB805D75DF1F910F91B7
:10032000FF90EF900895962F282F2053905340531D
:1003300084E6289F900111248AE0989FC00111242F
:10034000820F840F99270895522F282F205360532E
:10035000405350532A3008F027506A3008F0675055
:100360004A3008F047505A3008F057503327322FA0
:1003700022273295307F862F9927982F8827282B80
:10038000392B842F992744E0880F991F4A95E1F76C
:10039000282B392B852F9927822B932B089580B7F3
:1003A000846080BFA09AA19A8B98A2988A98A89AF4
:1003B000A99A85B78F78806285BF85B78D7F85BF05
:1003C00085B78E7F85BF85B7877F85BF85B78B7FD4
:1003D00085BF8BB78F7B8BBF8BB78F778BBF089514
:1003E00080915E0191E0892780935E0180915E019A
:1003F000882311F0A8980895A89A089580915D0126
:1004000091E0892780935D0180915D01882311F43B
:10041000A9980895A99A0895949881E090E03DDE06
:10042000949A81E090E039DE08951F9390915C01E9
:10043000992339F0839B51C09A9B4FC010925C0165
:100440004CC0839926C09093620180915B018230F9
:1004500049F080915701909158010196909358016D
:100460008093570120915701309158018091590193
:1004700090915A018217930730F481E090E09093B5
:1004800058018093570181E080935B0180935C0168
:1004900024C09A9922C09093620182E080935B010C
:1004A00090937A018091810190918201A0918301C2
:1004B000B091840180937D0190937E01A0937F0190
:1004C000B0938001A89A81E790E0EBDE11E01093F1
:1004D0006000A2DF949810935C011F910895DC01E5
:1004E000F894E199FECF1CDB802D7894992708952C
:1004F000DC01F894E199FECF062E1ADB789408957A
:1005000083E090E0ECDF80936101809161018F3F97
:1005100041F487ED809361016091610183E090E097
:10052000E7DF08958FB9779BFECF8FB199270895A4
:100530001F93CF93182FC0E0C81728F48FEFF2DF76
:10054000CF5FC117D8F3CF911F910895EF92FF921B
:100550000F931F93CF93C82F7A018B018064E2DF42
:10056000812F9927AA27BB27DDDFC801AA27BB2730
:10057000D9DFBB27A12F902F8F2DD4DF8E2DD2DF77
:100580008FEFCC2311F485E903C0C83009F487E864
:10059000C9DFCF911F910F91FF90EF9008951F93A6
:1005A000CF938EE58DB9C29A84E6C2DFC29881E00E
:1005B00090E073DD40E050E060E070E080E0C6DF96
:1005C00083E0B6DF81E090E068DD4AEA51E060E078
:1005D00070E088E0BBDF16E08FEFA4DF853021F408
:1005E00081E08093A80104C0813011F41092A80129
:1005F000115017FFF1CF81E090E04FDD10E040E0B7
:1006000050E060E070E087E3A1DF8FEF8BDF8FEFDA
:1006100089DFC82F8FEF86DF8AE090E03EDD40E083
:1006200050E060E070E489E291DF8FEF7BDF8FEFD5
:1006300079DFC80F8FEF76DF8AE090E02EDDCC23E4
:1006400019F01F5F1233D8F2CC2321F0C29A80E058
:1006500090E020C08091A8018823B1F440E050E0F0
:1006600060E070E08AE372DF8FEF5CDF8FEF5ADFCC
:100670008FEF58DFC82F83E05BDF8FEF53DFC6FDBE
:1006800003C081E08093A8018AE090E006DDC29A71
:1006900081E090E0CF911F9108950F931F93CF9326
:1006A000DF93EC01DB018A01A8958CE58DB980917F
:1006B000A801813039F489E0AA0FBB1FCC1FDD1FD0
:1006C0008A95D1F7C298AD01BE0181E13FDF8091EB
:1006D000AF01882329F08FEF25DF8093AF01F9CF99
:1006E0008091AF018E3F29F08FEF1CDF8093AF0127
:1006F000F9CFE80101501E4F8FEF14DF89930C17DB
:100700001D07D0F78FEF0EDF8FEF0CDF8AE010DFD1
:10071000C29ADF91CF911F910F9108950F931F936C
:10072000CF93DF93EC01DB018A01A8958CE58DB9AD
:100730008091A801813039F499E0AA0FBB1FCC1F2A
:10074000DD1F9A95D1F7C298AD01BE0188E1FEDEAA
:100750008091AF01882329F08FEFE4DE8093AF0111
:10076000F9CF8EEFDFDEE80101501E4F8991DADE0E
:100770000C171D07D8F78091AF0199278F719070E2
:10078000059741F08FEFCEDE8093AF0185E090E0DA
:1007900084DCF1CF8AE0CCDEC29ADF91CF911F9149
:1007A0000F9108958C9A8D9A8E9A8F98959A969A11
:1007B0000895F8DF31DE94980895FF920F931F9308
:1007C000F82E8B0181E58DB9959882E0ABDE8F2DF7
:1007D000A9DE812F9927A6DE802FA4DE959A1F918E
:1007E0000F91FF9008950F931F93182F81E58DB9F6
:1007F000959883E097DE812F95DE8FEF93DE992722
:10080000182F00278FEF8EDE9927959A802B912B3A
:100810001F910F9108952FEF322F381B832F261B26
:100820009927982F88273327822B932BBC018BE0A5
:10083000C4DF81E090E031DC0895AA27BB274AECB1
:1008400051E0BC01CD0129DF8091D501282F33274C
:100850008091D6019927982F8827282B392B309300
:10086000AA012093A9018091D7018093A1018091D1
:10087000D801282F33278091D9019927982F8827CD
:10088000282B392B8091550190915601280F391F43
:100890003093A3012093A2018091EA01282F3327EE
:1008A000442755278091EB019927AA27BB27BA2F08
:1008B000A92F982F8827282B392B4A2B5B2B809127
:1008C000EC019927AA27BB27DC0199278827282B29
:1008D000392B4A2B5B2B8091ED019927AA27BB2747
:1008E000B82FAA2799278827282B392B4A2B5B2B2F
:1008F0002093B0013093B1014093B2015093B30102
:100900008091EE01282F3327442755278091EF014E
:100910009927AA27BB27BA2FA92F982F8827282BDA
:10092000392B4A2B5B2B8091F0019927AA27BB27F3
:10093000DC0199278827282B392B4A2B5B2B8091A8
:10094000F1019927AA27BB27B82FAA27992788271B
:10095000282B392B4A2B5B2B2093AB013093AC0116
:100960004093AD015093AE018091F601282F3327BB
:10097000442755278091F7019927AA27BB27BA2F2B
:10098000A92F982F8827282B392B4A2B5B2B809156
:10099000F8019927AA27BB27DC0199278827282B4C
:1009A000392B4A2B5B2B8091F9019927AA27BB276A
:1009B000B82FAA2799278827282B392B4A2B5B2B5E
:1009C0002093A4013093A5014093A6015093A70161
:1009D0008091C803282F33278091C9039927982F26
:1009E0008827282B392B3093B5012093B401089523
:1009F000EF92FF920F931F93DC01CB01E090AB01CC
:100A0000F090AC010091AD011091AE01EE0CFF1C15
:100A1000001F111F0297A109B1092091A1013327DD
:100A200044275527BC01CD0148D8DC01CB01E80E95
:100A3000F91E0A1F1B1F8091A2019091A301AA27F2
:100A4000BB27E80EF91E0A1F1B1FC801B7011F9123
:100A50000F91FF90EF9008950F931F939B01AC01AE
:100A6000DC01CB018F779070A070B07072E0880FBE
:100A7000991FAA1FBB1F7A95D1F78C018091A20103
:100A80009091A301AA27BB2767E056954795379514
:100A900027956A95D1F7820F931FA41FB51F4AECC3
:100AA00051E0BC01CD01F9DDF801E653FE4F808134
:100AB000282F33274427552781819927AA27BB2729
:100AC000BA2FA92F982F8827282B392B4A2B5B2B3D
:100AD00082819927AA27BB27DC0199278827282B01
:100AE000392B4A2B5B2B83819927AA27BB27B82F49
:100AF000AA2799278827282B392B4A2B5B2BCA0139
:100B0000B9011F910F9108957F928F929F92AF929A
:100B1000BF92CF92DF92EF92FF920F931F93CF93EA
:100B2000DF935C01762E842E922EC02EE090A401DD
:100B3000F090A5010091A6011091A7018FEFE81692
:100B40008FEFF8068FEF08078FE0180709F46FC0E2
:100B5000DD248091A101D81608F063C0C801B70157
:100B600047DFDC01CB018D0D911DA11DB11D4AECAC
:100B700051E0BC01CD0191DD30E0EAECF1E040E074
:100B800050E08081882309F452C08085871509F0E0
:100B90003FC081858815E1F582858915C9F5838572
:100BA000C816B1F520E0E501DA01A653BE4F9D91CC
:100BB0008991981769F5273041F584899927AA27E3
:100BC000BB27AC013327222785899927AA27BB2772
:100BD000B82FAA2799278827282B392B4A2B5B2B3C
:100BE000828D9927AA27BB27282B392B4A2B5B2BD1
:100BF000838D9927AA27BB27BA2FA92F982F88273B
:100C0000282B392B4A2B5B2B16C02F5F283078F20C
:100C10003F5F405E5F4FB096303108F4B2CFD3945F
:100C200098CFC801B70118DF7B018C0187CF20E086
:100C300030E040E050E0CA01B901DF91CF911F914F
:100C40000F91FF90EF90DF90CF90BF90AF909F906B
:100C50008F907F9008952F923F924F925F926F9264
:100C60007F928F929F92AF92BF92CF92DF92EF923C
:100C7000FF920F931F93CF93DF93CDB7DEB72697E5
:100C80000FB6F894DEBF0FBECDBFDC01CB011A0159
:100C900029830A83EB82CC822501662477247C0198
:100CA0008D018FEFE8168FEFF8068FEF08078FE0C2
:100CB000180709F49CC0AA248091A101A81608F085
:100CC0008BC0C801B70194DEDC01CB018A0D911DF8
:100CD000A11DB11D4AEC51E0BC01CD01DEDC99241F
:100CE000EAECF1E0CC24DD248081882309F47FC084
:100CF000853E09F464C080859981891709F05FC039
:100D00008185AA818A1709F05AC08285BB818B1719
:100D100009F055C083859C81981709F050C008944C
:100D2000611C711CBB24B81408F049C0282D33275E
:100D300021503040B101D601A653BE4FBE83AD83D2
:100D400040E050E0AD81BE819D91BE83AD83DB016B
:100D50008D91BD01981799F54217530759F5D201A6
:100D60006D927C9284899927AA27BB27AC013327EF
:100D7000222785899927AA27BB27B82FAA27992731
:100D80008827282B392B4A2B5B2B828D9927AA2762
:100D9000BB27282B392B4A2B5B2B838D9927AA271E
:100DA000BB27BA2FA92F982F8827282B392B4A2BFE
:100DB0005B2B21C0B3944F5F5F4FB81418F293942C
:100DC00080E290E0C80ED91EE80FF91F9FE0991548
:100DD00008F08ACFA39470CFC801B7013DDE7B0134
:100DE0008C016F5F7F4F8F4F9F4009F064CF20E0F1
:100DF00030E040E050E0CA01B90126960FB6F89401
:100E0000DEBF0FBECDBFDF91CF911F910F91FF903D
:100E1000EF90DF90CF90BF90AF909F908F907F909A
:100E20006F905F904F903F902F9008957F928F9298
:100E30009F92AF92BF92CF92DF92EF92FF920F9369
:100E40001F93CF93DF93DC01CB015A01722E802ECA
:100E50009E2CC0E0D0E07C018D018FEFE8168FEF73
:100E6000F8068FEF08078FE0180709F462C0DD2449
:100E70008091A101D81608F056C0C801B701B8DDAD
:100E8000DC01CB018D0D911DA11DB11D4AEC51E07E
:100E9000BC01CD0102DC90E0EAECF1E08081882326
:100EA00009F447C0853EC1F180858715A9F5818584
:100EB000881591F58285891579F58385C81661F5C0
:100EC0002196CA15DB0541F584899927AA27BB27F6
:100ED000AC013327222785899927AA27BB27B82F5A
:100EE000AA2799278827282B392B4A2B5B2B828D01
:100EF0009927AA27BB27282B392B4A2B5B2B838DBD
:100F00009927AA27BB27BA2FA92F982F8827282BE4
:100F1000392B4A2B5B2B11C09F5FB096903108F4A0
:100F2000BDCFD394A5CFC801B70196DD7B018C015D
:100F300094CF20E030E040E050E0CA01B901DF91F9
:100F4000CF911F910F91FF90EF90DF90CF90BF90C6
:100F5000AF909F908F907F9008952F923F924F92E5
:100F60005F926F927F928F929F92AF92BF92CF9239
:100F7000DF92EF92FF920F931F93CF93DF93CDB742
:100F8000DEB723970FB6F894DEBF0FBECDBFDC01EE
:100F9000CB014983222E302E4E2C662477247C01EF
:100FA0008D018FEFE8168FEFF8068FEF08078FE0BF
:100FB000180709F46EC0AA248091A101A81608F0B0
:100FC0005DC0C801B70114DDDC01CB018A0D911DA4
:100FD000A11DB11D4AEC51E0BC01CD015EDB5524E1
:100FE000882499249AECC92E91E0D92EF6018081AB
:100FF000882339F470925A016092590181E090E09F
:101000004EC0853E71F1F6018085F9818F1749F553
:10101000F6018185821529F58285831511F5838571
:101020004816F9F40894611C711C80915F018823B3
:10103000C1F0C30144D988E790E033D987E0B82EE6
:10104000C40186539E4F9B838A83EA81FB818191F1
:10105000FB83EA83D8D8BA94B7FEF7CF8BE790E04A
:1010600020D9539480E290E0C80ED91E880E991EB4
:101070009FE0951508F0BACFA3949ECFC801B701A1
:10108000EBDC7B018C016F5F7F4F8F4F9F4009F03E
:1010900092CF70925A016092590180E090E02396BD
:1010A0000FB6F894DEBF0FBECDBFDF91CF911F9179
:1010B0000F91FF90EF90DF90CF90BF90AF909F90F7
:1010C0008F907F906F905F904F903F902F900895FA
:1010D0008F92AF92BF92CF92EF920F93FC01862E28
:1010E000109262018091490190914A01A0914B01B7
:1010F000B0914C010097A105B105B9F12130B9F4C7
:101100008091490190914A01A0914B01B0914C010D
:1011100067E5A62E61E0B62E50E2C52E43E3E42E2D
:1011200000E52DE4AF01BC01CD0195DD13C02230F7
:10113000F9F48091490190914A01A0914B01B0913D
:101140004C0130E2C32E23E3E22E00E52DE4BC0186
:10115000CD016CDEDC01CB018093510190935201F3
:10116000A0935301B093540103C081E090E063C0A9
:101170008091510190915201A0915301B09154017D
:101180000097A105B10519F482E090E054C0809168
:10119000510190915201A0915301B0915401BC01B1
:1011A000CD0126DCDC01CB0180934D0190934E01F3
:1011B000A0934F01B093500180914D0190914E0149
:1011C000A0914F01B09150014AEC51E0BC01CD011A
:1011D00064DA10924801109247011092460181E0B2
:1011E0008093620180937A018EE790E05AD88091D3
:1011F00057019091580163D88BE790E052D88091C5
:101200006000813019F41092600006D964E078E043
:1012100080E0D3DA81E090E040D760E070EC83E0DA
:10122000CCDA81E090E039D7609161018091610171
:10123000F2DA80E090E00F91EF90CF90BF90AF9006
:101240008F9008951F93CF93DF938091620188233D
:1012500009F4BDC0879BBBC09698C0E0D0E01FE1F9
:10126000E0914701F091480175E0EE0FFF1F7A957C
:10127000E1F7EC0FFD1FE653FE4F808153D911506B
:10128000219617FFEDCF969A8091470190914801E2
:101290000196909348018093470180914701909176
:1012A0004801409749F510924801109247018091FA
:1012B0004D0190914E01A0914F01B09150010196C6
:1012C000A11DB11D80934D0190934E01A0934F013C
:1012D000B093500180914D0190914E01A0914F012A
:1012E000B09150014AEC51E0BC01CD01D6D98091BA
:1012F00046018F5F80934601909146018091A10144
:10130000981708F462C010924601809151019091A3
:101310005201A0915301B0915401BC01CD019CDB5D
:10132000DC01CB018093510190935201A0935301B2
:10133000B09354018091510190915201A0915301B9
:10134000B09154018F5F9F4FAF4FBF40E1F41092B7
:101350006201809157019091580101969093580134
:10136000809357012091590130915A01281739076C
:1013700030F481E090E0909358018093570181E030
:1013800080935B0124C08091510190915201A09102
:101390005301B0915401BC01CD012ADBDC01CB012A
:1013A00080934D0190934E01A0934F01B093500153
:1013B00080914D0190914E01A0914F01B09150014B
:1013C0004AEC51E0BC01CD0168D9879945CFDF9146
:1013D000CF911F91089520E0261768F4FC01A6EB39
:1013E000B1E09D918191981719F080E090E0089507
:1013F0002F5F2617B0F381E090E0089580916C0193
:10140000882309F485C026D780916C0180936B01F5
:1014100010926C0166E084E890E0DDDF882319F02B
:1014200081E090E0089566E08BE890E0D4DF8823C7
:1014300019F082E090E0089565E082E990E0CBDF6A
:10144000882319F083E090E0089564E088E990E053
:10145000C2DF882319F084E090E0089564E08DE90C
:1014600090E0B9DF882319F085E090E0089564E00A
:1014700082EA90E0B0DF882319F086E090E00895DA
:1014800067E087EA90E0A7DF882319F08BE090E01F
:10149000089565E08FEA90E09EDF882319F08CE0E4
:1014A00090E0089568E085EB90E095DF882319F0DF
:1014B0008DE090E0089564E08EEB90E08CDF88236F
:1014C00019F08EE090E0089565E083EC90E083DF12
:1014D000882319F085E190E0089566E089EC90E0BA
:1014E0007ADF882319F086E190E0089566E080EDC8
:1014F00090E071DF882319F087E190E0089567E0BC
:1015000087ED90E068DF882319F08FE190E008957F
:1015100080E090E00895EF920F931F93CF93DF93B5
:101520006DDF9927AA27BB27FC013197EF31F10521
:1015300008F056C1ED5EFF4F099410926201809150
:101540005B01823049F080915701909158010196DA
:101550009093580180935701209157013091580181
:101560008091590190915A0182179307F0F481E01C
:1015700090E017C01092620180915701909158013C
:10158000009729F00197909358018093570180911B
:10159000570190915801892B41F480915901909104
:1015A0005A01909358018093570181E080935B0129
:1015B00017C11092620183E080935B0180916B01FF
:1015C000855021E040E050E0682F8BEB91E080DD1A
:1015D00007C1809162018823C1F0109262011092CC
:1015E0007A018091810190918201A0918301B09153
:1015F000840180937D0190937E01A0937F01B0933D
:101600008001A8988FED90E0EAC080915B01833063
:1016100009F0E6C081E08093620180937A0186EE52
:1016200090E0DDC01092620182E080935B01109235
:101630007A018091810190918201A0918301B09102
:10164000840180937D0190937E01A0937F01B093EC
:101650008001A89A81E790E024D681E08093600021
:10166000DBD69498BDC081E080935F0180914901F1
:1016700090914A01A0914B01B0914C01E0E2EE2E15
:1016800003E320E54DE4BC01CD0167DCA9C0409136
:10169000BF016091BE018091BD0145D6809361017B
:1016A00020C02091BE014091BD016091BC0180919C
:1016B000BB014AD6BC0182E080D881E090E0EDD445
:1016C0008DEE90E08CC08091BE018C3411F460E00E
:1016D0000AC0823521F46091610180E006C08D343A
:1016E00079F7609161018091610195D8E9CF6091AE
:1016F000610183E090E0FCD6E3CF8DEE90E0D1D5A0
:1017000088E190E02CE00FB6F894A89581BD0FBE5B
:1017100021BDFFCF4091BE016091BD018091BC0110
:1017200002D69927AA27BB27BC01CD0120E737E1C4
:1017300040E050E0C2D1DC01CB0106EF1BE09C0190
:10174000AD0161E070E082E036D5BACFF894A89A96
:10175000A99A62D6949888E10FB6F89481BD11BC1D
:101760000FBE83EF90E09DD585E090E096D48BB7D7
:1017700080688BBF789485B7806885BF889585B76A
:101780008F7785BF49D62CC02091C0014091BF0101
:101790006091BE018091BD01D7D5AA27BB274AEC35
:1017A00051E0BC01CD0179D700E010E0CAECD1E0F6
:1017B000C8018F709070892B41F48BE790E071D550
:1017C000C8017DD580E091E06CD5899157D50F5F38
:1017D0001F4F82E00030180758F38BE790E061D587
:1017E000DF91CF911F910F91EF90089581E0809349
:1017F00060010895809160018823F9F0F8941092B7
:101800006001A89AA99A08D6949888E10FB6F8942E
:1018100081BD11BC0FBE84E091E043D585E090E02E
:101820003CD48BB780688BBF789485B7806885BFC0
:10183000889585B78F7785BFEFD50895829B1DC0AA
:10184000F894A89AA99AE8D5949888E10FB6F894E4
:1018500081BD11BC0FBE81E191E023D585E090E010
:101860001CD48BB780648BBF789485B7806885BFA4
:10187000889585B78F7785BF0895A99885B78D7F9F
:1018800085BF85B7816085BF8BB780648BBF0895A6
:10189000CFE5D4E0DEBFCDBF88E190E02DE00FB60C
:1018A000F894A89581BD0FBE21BD79D5A7D4579ACC
:1018B0008CE287BB88BB24D67CD7C0DFA8956FD6C7
:1018C000882309F4FFCF8CE191E0EBD4A89580E068
:1018D00090E0B3D78091B4019091B50185559A4AB3
:1018E00061F48091A9019091AA018050924029F45D
:1018F00010925601109255011EC0809191039927B4
:10190000982F8827209190033327822B932B909335
:1019100056018093550191D78091B4019091B50102
:1019200085559A4A39F48091A9019091AA01805075
:10193000924009F0FFCF88E291E0B3D48091560144
:101940009DD4809155019AD48BE790E0AAD400E110
:1019500020E2422F622F81E391E0D6D8DC01CB0157
:101960008093490190934A01A0934B01B0934C019D
:1019700010925F018091490190914A01A0914B0121
:10198000B0914C01F0E2EF2E03E320E54DE4BC0101
:10199000CD01E3DA8AE391E084D4809159019091FA
:1019A0005A018DD48BE790E07CD491D305E112E00D
:1019B0002AE030E040E050E06FEF7FEF80E0FBD3C3
:1019C00000EF11E028E230E040E050E06FEF7FEF01
:1019D00081E0F1D310927A0180918101909182018E
:1019E000A0918301B091840180937D0190937E0149
:1019F000A0937F01B093800188E190E02FE00FB6C3
:101A0000F894A89581BD0FBE21BD7894A8958299C0
:101A1000FDCF80915B018130D1F4C3E0C0935B01C5
:101A200022E0409157015091580160E083E691E037
:101A30004FDB882361F010925D010EEF11E024E18D
:101A400030E040E050E066E070E08C2FB4D363DD1E
:101A5000F9DBD0DEDBCF1F920F920FB60F9211246D
:101A60002F938F939F938BB78F7B8BBF88E190E0F1
:101A70002CE00FB6F894A89581BD0FBE21BDFFCF15
:101A80001F920F920FB60F9211242F938F939F9353
:101A90008BB78F778BBFA99888E190E02FE00FB6C6
:101AA000F894A89581BD0FBE21BD9F918F912F9174
:101AB0000F900FBE0F901F901895629FD001739FDB
:101AC000F001829FE00DF11D649FE00DF11D929FDA
:101AD000F00D839FF00D749FF00D659FF00D992719
:101AE000729FB00DE11DF91F639FB00DE11DF91F3D
:101AF000BD01CF0111240895AA1BBB1B51E107C0F2
:101B0000AA1FBB1FA617B70710F0A61BB70B881F8D
:101B1000991F5A95A9F780959095BC01CD0108951C
:101B2000E199FECFBFBBAEBBE09A11960DB208950E
:101B3000E199FECFBFBBAEBB0DBA11960FB6F894BC
:081B4000E29AE19A0FBE08953C
:101B48000130313233343536373839414243444530
:101B58004653544F500D0A002E20000D0A00504CD9
:101B680041595F00706C61793E3E00706C61793C50
:101B78003C00706C61795F00686F6C640073746F0F
:101B880070006C69737400766F6C756D655F0062C8
:101B98006173735F0062616C616E63655F0073619E
:101BA800766500726573657400736C6565705F00B7
:101BB8007077646F776E00736563746F725F004847
:101BC8004F4C440D0A00504C41590D0A0041434BFB
:101BD8000D0A00504F57455220444F574E0D0A00EA
:101BE800203A2000534C45455020444F574E0D0A8B
:101BF80000534420454D5054590D0A005344204980
:101C08004E534552540D0A004D4252203D0930783A
:101C1800004D50335F46494C45004D50335F4649AF
:061C28004C45203A2000AB
:00000001FF
